:020000040000FA
:0408000016EF09F0F6
:1008100003B26CEF05F0F2B48AEF05F09EB092EFF0
:1008200005F09EB29AEF05F0F2A81AEF04F0F2B2CA
:100830001CEF04F0C5EF08F0CD90F2929EA026EFD9
:1008400004F00101533F26EF04F0542BAEC1B2F186
:10085000AFC1B3F1B0C1B4F1B1C1B5F1AAC1AEF14C
:10086000ABC1AFF1ACC1B0F1ADC1B1F1A6C1AAF15C
:10087000A7C1ABF1A8C1ACF1A9C1ADF1A2C1A6F16C
:10088000A3C1A7F1A4C1A8F1A5C1A9F19EC1A2F17C
:100890009FC1A3F1A0C1A4F1A1C1A5F19AC19EF18C
:1008A0009BC19FF19CC1A0F19DC1A1F196C19AF19C
:1008B00097C19BF198C19CF199C19DF1CECF96F162
:1008C000CFCF97F153C198F154C199F1CF6ACE6A55
:1008D0000101536B546B9E90CD800FBC0F8E0FBAED
:1008E00075EF04F00F8AC5EF08F00F8C0FBEB1EF63
:1008F00004F096C19AF197C19BF198C19CF199C1FE
:100900009DF19AC19EF19BC19FF19CC1A0F19DC137
:10091000A1F19EC1A2F19FC1A3F1A0C1A4F1A1C107
:10092000A5F1A2C1A6F1A3C1A7F1A4C1A8F1A5C1D7
:10093000A9F1A6C1AAF1A7C1ABF1A8C1ACF1A9C1A7
:10094000ADF1AAC1AEF1ABC1AFF1ACC1B0F1ADC177
:10095000B1F1AEC1B2F1AFC1B3F1B0C1B4F1B1C147
:10096000B5F101015E6B5F6B606B616B96515E2749
:1009700097515F2398516023995161239A515E27C3
:100980009B515F239C5160239D5161239E515E27A3
:100990009F515F23A0516023A1516123A2515E2783
:1009A000A3515F23A4516023A5516123A6515E2763
:1009B000A7515F23A8516023A9516123AA515E2743
:1009C000AB515F23AC516023AD516123AE515E2723
:1009D000AF515F23B0516023B1516123B2515E2703
:1009E000B3515F23B4516023B5516123D890010105
:1009F000613360335F335E33D8900101613360331C
:100A00005F335E33D8900101613360335F335E330F
:100A100000C10CF101C10DF102C10EF103C10FF1D2
:100A200004C110F105C111F106C112F107C113F1A2
:100A300008C114F109C115F10AC116F10BC117F172
:100A400034C135F111B830EF05F00101620E046FC9
:100A5000010E056F000E066F000E076F39EF05F0EF
:100A60000101A70E046F020E056F000E066F000E47
:100A7000076F5EC100F15FC101F160C102F161C1A8
:100A800003F1F7EC18F003BF48EF05F011B6108C36
:100A900011A050EF05F010BA50EF05F00F80108A4A
:100AA0000CC100F10DC101F10EC102F10FC103F142
:100AB00010C104F111C105F112C106F113C107F112
:100AC00014C108F115C109F116C10AF117C10BF1E2
:100AD00035C134F1C5EF08F00392ABB2AB98AB88E7
:100AE000030103EE00F080517F0BE92604C0EFFF05
:100AF000802B8151805D700BD8A48B8200008051C7
:100B0000815D700BD8A48B9281518019D8B4079065
:100B1000C5EF08F0F2940101453FC5EF08F0462B00
:100B2000C5EF08F09E900101533FC5EF08F0542B2C
:100B3000C5EF08F09E9211B800EF07F08BB4A8EF54
:100B400005F010ACA8EF05F08B84109CA9EF05F020
:100B50008B94C3CF55F1C4CF56F1C28207B413EFC3
:100B600006F047C14BF148C14CF149C14DF14AC1B2
:100B70004EF15EC162F15FC163F160C164F161C1B8
:100B800065F196C1B6F197C1B7F198C1B8F199C1B5
:100B9000B9F19AC1BAF19BC1BBF19CC1BCF19DC135
:100BA000BDF19EC1BEF19FC1BFF1A0C1C0F1A1C105
:100BB000C1F1A2C1C2F1A3C1C3F1A4C1C4F1A5C1D5
:100BC000C5F1A6C1C6F1A7C1C7F1A8C1C8F1A9C1A5
:100BD000C9F1AAC1CAF1ABC1CBF1ACC1CCF1ADC175
:100BE000CDF1AEC1CEF1AFC1CFF1B0C1D0F1B1C145
:100BF000D1F1B2C1D2F1B3C1D3F1B4C1D4F1B5C115
:100C0000D5F1010155515B2756515C23E86A5D23FC
:100C10000E2E13EF06F05CC157F15DC158F15B6B0E
:100C20005C6B5D6B078E0201002FC5EF08F03C0E78
:100C3000006F11BA108E00C10CF101C10DF102C19B
:100C40000EF103C10FF104C110F105C111F106C18C
:100C500012F107C113F108C114F109C115F10AC15C
:100C600016F10BC117F134C135F101018A6740EF6C
:100C700006F08B6740EF06F08C6740EF06F08D675B
:100C800044EF06F074EF06F08EC100F18FC101F160
:100C900090C102F191C103F10101010E046F000E38
:100CA000056F000E066F000E076FF7EC18F000C11D
:100CB0008EF101C18FF102C190F103C191F1006782
:100CC00069EF06F0016769EF06F0026769EF06F069
:100CD000036774EF06F08AC18EF18BC18FF18CC16E
:100CE00090F18DC191F10F80D57ED5BE6BD0D6CF5E
:100CF00047F1D7CF48F145C149F1E86AE8CF4AF159
:100D000011B6108C109047C100F148C101F149C1E2
:100D100002F14AC103F101010A0E046F000E056FD2
:100D2000000E066F000E076FF7EC18F003AF10808F
:100D3000010154A7A8EF06F00F9A0F9C0F9E010126
:100D4000000E5E6F600E5F6F3D0E606F080E616F8C
:100D5000010147BFB8EF06F04867B8EF06F04967F2
:100D6000B8EF06F04A67B8EF06F0F288DDEF06F05C
:100D7000F2985E6B5F6B606B616B966B976B986BB9
:100D8000996B9A6B9B6B9C6B9D6B9E6B9F6BA06B27
:100D9000A16BA26BA36BA46BA56BA66BA76BA86BD7
:100DA000A96BAA6BAB6BAC6BAD6BAE6BAF6BB06B87
:100DB000B16BB26BB36BB46BB56BD76AD66A01011A
:100DC000456B466B0CC100F10DC101F10EC102F182
:100DD0000FC103F110C104F111C105F112C106F1F7
:100DE00013C107F114C108F115C109F116C10AF1C7
:100DF00017C10BF135C134F1C5EF08F0C5EF08F0AC
:100E00000201002F4EEF08F0D59ED6CF47F1D7CF85
:100E100048F145C149F1E86AE8CF4AF1D76AD66A94
:100E20000101456B466BD58E11BA108E00C10CF1D5
:100E300001C10DF102C10EF103C10FF104C110F1A6
:100E400005C111F106C112F107C113F108C114F176
:100E500009C115F10AC116F10BC117F134C135F101
:100E60000FA0109A11B840EF07F00101620E046F55
:100E7000010E056F000E066F000E076F49EF07F0B9
:100E80000101A70E046F020E056F000E066F000E23
:100E9000076F47C100F148C101F149C102F14AC1E0
:100EA00003F1F7EC18F003BF5AEF07F011B6108CFE
:100EB00011B00F800CC100F10DC101F10EC102F1A2
:100EC0000FC103F110C104F111C105F112C106F106
:100ED00013C107F114C108F115C109F116C10AF1D6
:100EE00017C10BF135C134F102013C0E006F00C196
:100EF0000CF101C10DF102C10EF103C10FF104C1EA
:100F000010F105C111F106C112F107C113F108C1B9
:100F100014F109C115F10AC116F10BC117F134C161
:100F200035F101018A679CEF07F08B679CEF07F0B2
:100F30008C679CEF07F08D67A0EF07F0D0EF07F00C
:100F40008EC100F18FC101F190C102F191C103F195
:100F50000101010E046F000E056F000E066F000EFA
:100F6000076FF7EC18F000C18EF101C18FF102C1DB
:100F700090F103C191F10067C5EF07F00167C5EF7C
:100F800007F00267C5EF07F00367D0EF07F08AC1EB
:100F90008EF18BC18FF18CC190F18DC191F10F80D9
:100FA000109047C100F148C101F149C102F14AC1A5
:100FB00003F101010A0E046F000E056F000E066FAB
:100FC000000E076FF7EC18F003AF1080010154A773
:100FD000F6EF07F00F9A0F9C0F9E0101000E5E6F57
:100FE000600E5F6F3D0E606F080E616F47C100F1CC
:100FF00048C101F149C102F14AC103F10101140ED6
:10100000046F050E056F000E066F000E076FF7ECFC
:1010100018F003AF0FEF08F0F28834EF08F0F29801
:101020005E6B5F6B606B616B966B976B986B996B8C
:101030009A6B9B6B9C6B9D6B9E6B9F6BA06BA16B6C
:10104000A26BA36BA46BA56BA66BA76BA86BA96B1C
:10105000AA6BAB6BAC6BAD6BAE6BAF6BB06BB16BCC
:10106000B26BB36BB46BB56B0CC100F10DC101F188
:101070000EC102F10FC103F110C104F111C105F15C
:1010800012C106F113C107F114C108F115C109F12C
:1010900016C10AF117C10BF135C134F18BB458EF09
:1010A00008F010AC58EF08F08B84109C59EF08F052
:1010B0008B94C3CF55F1C4CF56F1C28207B4C3EFAE
:1010C00008F047C14BF148C14CF149C14DF14AC14B
:1010D0004EF15EC162F15FC163F160C164F161C153
:1010E00065F196C1B6F197C1B7F198C1B8F199C150
:1010F000B9F19AC1BAF19BC1BBF19CC1BCF19DC1D0
:10110000BDF19EC1BEF19FC1BFF1A0C1C0F1A1C19F
:10111000C1F1A2C1C2F1A3C1C3F1A4C1C4F1A5C16F
:10112000C5F1A6C1C6F1A7C1C7F1A8C1C8F1A9C13F
:10113000C9F1AAC1CAF1ABC1CBF1ACC1CCF1ADC10F
:10114000CDF1AEC1CEF1AFC1CFF1B0C1D0F1B1C1DF
:10115000D1F1B2C1D2F1B3C1D3F1B4C1D4F1B5C1AF
:10116000D5F1010155515B2756515C23E86A5D2397
:101170000E2EC3EF08F05CC157F15DC158F15B6BF7
:101180005C6B5D6B078EC5EF08F002C0E0FF00509E
:1011900001C0D8FF1000A6B2CBEF08F00CC0A9FF29
:1011A0000BC0A8FFA69EA69CA684F29E550EA76E15
:1011B000AA0EA76EA682F28EA694A6B2DDEF08F064
:1011C0000C2A1200A96EA69EA69CA680A8500C2AE6
:1011D000120004012C0E826FC5EC0AF0F2EC19F03B
:1011E0000C50E2EC08F0E8CF00F10C50E2EC08F013
:1011F000E8CF01F101AF02EF09F00101FF0E026F2C
:10120000FF0E036F95EC19F029670EEF09F004014A
:10121000200E826FC5EC0AF013EF09F004012D0EC9
:10122000826FC5EC0AF0BFEC17F01200076A0F6A74
:10123000106A116A0F010E0EC16E860EC06E030E8B
:10124000C26E0F01896A110E926E080E8A6EF10E3F
:10125000936E8B6A800E946EF18EFC0EE2EC08F0B9
:10126000E8CF0BF00BA011800BA211820BA411840C
:101270000BA611860BA811880BAA118A0E6A010110
:101280005B6B5C6B5D6B576B586BF29A0101476B44
:10129000486B496B4A6B4B6B4C6B4D6B4E6B4F6B9A
:1012A000506B516B526B456B466BD76AD66A0F0118
:1012B000280ED56EF28A9D90B00ECD6E01015E6B48
:1012C0005F6B606B616B626B636B646B656B666BB2
:1012D000676B686B696B536B546BCF6ACE6A0F9AFE
:1012E0000F9C0F9E9D80760ECA6E9D8202013C0E61
:1012F000006FCC6A160EE2EC08F0E8CF00F1170E92
:10130000E2EC08F0E8CF01F1180EE2EC08F0E8CFCB
:1013100002F1190EE2EC08F0E8CF03F1010103AF8E
:10132000ACEF09F0F2EC19F0160E0C6E00C10BF0E8
:10133000CBEC08F0170E0C6E01C10BF0CBEC08F0F3
:10134000180E0C6E02C10BF0CBEC08F0190E0C6EEF
:1013500003C10BF0CBEC08F000C18AF101C18BF1A5
:1013600002C18CF103C18DF100C18EF101C18FF179
:1013700002C190F103C191F11A0EE2EC08F0E8CF3E
:1013800000F11B0EE2EC08F0E8CF01F11C0EE2ECDC
:1013900008F0E8CF02F11D0EE2EC08F0E8CF03F10F
:1013A000010103AF02EF0AF0F2EC19F01A0E0C6E15
:1013B00000C10BF0CBEC08F01B0E0C6E01C10BF062
:1013C000CBEC08F01C0E0C6E02C10BF0CBEC08F05D
:1013D0001D0E0C6E03C10BF0CBEC08F01A0EE2EC04
:1013E00008F0E8CF00F11B0EE2EC08F0E8CF01F1C5
:1013F0001C0EE2EC08F0E8CF02F11D0EE2EC08F062
:10140000E8CF03F100C192F101C193F102C194F15F
:1014100003C195F1240EAC6E900EAB6E240EAC6E33
:10142000080EB86E000EB06E1F0EAF6E0401806B1A
:10143000816B0F01900EAB6E0F019D8A0301806BD3
:10144000816BC26B8B92B8EC1AF007900001F28EA0
:10145000F28C07B06CEF16F00FB008EF11F010BE71
:1014600008EF11F00301805181197F0BD8B46CEFA4
:1014700016F013EE00F081517F0BE126812BE7CFB0
:10148000E8FFE00BD8B46CEF16F023EE82F0C25107
:101490003F0BD926E7CFDFFFC22BDF50780AD8A455
:1014A0006CEF16F007808EC100F18FC101F190C181
:1014B00002F191C103F10101040E046F000E056FEA
:1014C000000E066F000E076FF7EC18F000AF72EF1A
:1014D0000AF00101030E8E6F000E8F6F000E906FE9
:1014E000000E916F03018251720AD8B408EF11F017
:1014F0008251520AD8B408EF11F08251750AD8B45B
:1015000008EF11F08251630AD8B426EF13F082512C
:10151000690AD8B4B5EF0DF082517A0AD8B4C8EF91
:101520000EF08251490AD8B454EF0DF08251500A9E
:10153000D8B472EF0CF08251700AD8B4B5EF0CF049
:101540008251540AD8B4E0EF0CF08251740AD8B436
:1015500026EF0DF082516D0AD8B4CAEF0BF082511C
:101560004D0AD8B4E3EF0BF08251730AD8B438EFC8
:1015700010F08251530AD8B49DEF10F08251590AED
:10158000D8B4D9EF0AF05DEF13F0040114EE00F0C7
:1015900080517F0BE12682C4E7FF802B12000401FB
:1015A0000D0E826FC5EC0AF00A0E826FC5EC0AF0D0
:1015B0001200FC0EE2EC08F0E8CF0BF003018351BF
:1015C000520AD8B428EF0BF003018351720AD8B441
:1015D0002BEF0BF003018351500AD8B42EEF0BF020
:1015E00003018351700AD8B431EF0BF0030183512A
:1015F000550AD8B434EF0BF003018351750AD8B4FF
:1016000037EF0BF0030183514C0AD8B43AEF0BF0DB
:10161000030183516C0AD8B43DEF0BF003018351F1
:10162000430AD8B440EF0BF003018351630AD8B4E6
:1016300043EF0BF003018351440AD8B446EF0BF09B
:1016400003018351640AD8B449EF0BF052EF0BF059
:101650000B904CEF0BF00B804CEF0BF00B924CEF20
:101660000BF00B824CEF0BF00B944CEF0BF00B8458
:101670004CEF0BF00B964CEF0BF00B864CEF0BF096
:101680000B984CEF0BF00B884CEF0BF00B9A4CEFD8
:101690000BF00B8A4CEF0BF0FC0E0C6E0BC00BF03A
:1016A000CBEC08F00401590E826FC5EC0AF01190E2
:1016B0001192119411961198119AFC0EE2EC08F017
:1016C000E8CF0BF00BA011800BA211820BA41184A8
:1016D0000BA611860BA811880BAA118A11A078EF0E
:1016E0000BF00401520E826FC5EC0AF07DEF0BF097
:1016F0000401720E826FC5EC0AF011A687EF0BF0A1
:1017000004014C0E826FC5EC0AF08CEF0BF0040163
:101710006C0E826FC5EC0AF011A896EF0BF0040175
:10172000430E826FC5EC0AF09BEF0BF00401630ED1
:10173000826FC5EC0AF011A2A5EF0BF00401500E68
:10174000826FC5EC0AF0AAEF0BF00401700E826FF5
:10175000C5EC0AF011A4B4EF0BF00401550E826F32
:10176000C5EC0AF0B9EF0BF00401750E826FC5EC01
:101770000AF011AAC3EF0BF00401440E826FC5EC0E
:101780000AF0C8EF0BF00401640E826FC5EC0AF09A
:101790005BEF13F004016D0E826FC5EC0AF00301DC
:1017A0008351300AD8B422EF0CF003018351310A7F
:1017B000D8B435EF0CF003018351320AD8B448EFA6
:1017C0000CF05DEF13F004014D0E826FC5EC0AF0D2
:1017D00033EC1AF084C331F185C332F186C333F19F
:1017E0000101296B40EC1AF0B7EC19F003018351A9
:1017F000300AD8B40AEF0CF003018351310AD8B48F
:1018000012EF0CF003018351320AD8B41AEF0CF036
:101810005DEF13F0FD0E0C6E00C10BF0CBEC08F089
:1018200022EF0CF0FE0E0C6E00C10BF0CBEC08F0BA
:1018300035EF0CF0FF0E0C6E00C10BF0CBEC08F096
:1018400048EF0CF00401300E826FC5EC0AF0040181
:101850002C0E826FC5EC0AF0F2EC19F0FD0EE2ECF2
:1018600008F0E8CF00F159EF0CF00401310E826F5F
:10187000C5EC0AF004012C0E826FC5EC0AF0F2EC04
:1018800019F0FE0EE2EC08F0E8CF00F159EF0CF091
:101890000401320E826FC5EC0AF0F2EC19F004017B
:1018A0002C0E826FC5EC0AF0FF0EE2EC08F0E8CFD8
:1018B00000F195EC19F031C182F40401300E822759
:1018C000C5EC0AF032C182F40401300E8227C5EC67
:1018D0000AF033C182F40401300E8227C5EC0AF00D
:1018E0005BEF13F083C32AF184C32BF185C32CF182
:1018F00086C32DF187C32EF188C32FF189C330F140
:101900008AC331F18BC332F18CC333F1010140EC56
:101910001AF0B7EC19F0160E0C6E00C10BF0CBEC00
:1019200008F0170E0C6E01C10BF0CBEC08F0180E8E
:101930000C6E02C10BF0CBEC08F0190E0C6E03C15B
:101940000BF0CBEC08F000C18AF101C18BF102C1B0
:101950008CF103C18DF100C18EF101C18FF102C183
:1019600090F103C191F154EF0DF083C32AF184C3C8
:101970002BF185C32CF186C32DF187C32EF188C3CB
:101980002FF189C330F18AC331F18BC332F18CC39B
:1019900033F1010140EC1AF0B7EC19F000C18AF103
:1019A00001C18BF102C18CF103C18DF100C18EF137
:1019B00001C18FF102C190F103C191F154EF0DF01B
:1019C00083C32AF184C32BF185C32CF186C32DF187
:1019D00087C32EF188C32FF189C330F18AC331F157
:1019E0008CC332F18DC333F1010140EC1AF0B7EC36
:1019F00019F00101000E046F000E056F010E066F55
:101A0000000E076F08EC19F01A0E0C6E00C10BF0F7
:101A1000CBEC08F01B0E0C6E01C10BF0CBEC08F008
:101A20001C0E0C6E02C10BF0CBEC08F01D0E0C6E00
:101A300003C10BF0CBEC08F000C192F101C193F1AE
:101A400002C194F103C195F154EF0DF083C32AF163
:101A500084C32BF185C32CF186C32DF187C32EF1EE
:101A600088C32FF189C330F18AC331F18CC332F1BD
:101A70008DC333F1010140EC1AF0B7EC19F001010C
:101A8000000E046F000E056F010E066F000E076F4B
:101A900008EC19F000C192F101C193F102C194F177
:101AA00003C195F154EF0DF0160EE2EC08F0E8CF0B
:101AB00000F1170EE2EC08F0E8CF01F1180EE2ECAD
:101AC00008F0E8CF02F1190EE2EC08F0E8CF03F1DC
:101AD00095EC19F078EC17F00401730E826FC5ECE9
:101AE0000AF004012C0E826FC5EC0AF08AC100F1E5
:101AF0008BC101F18CC102F18DC103F195EC19F09C
:101B000078EC17F00401730E826FC5EC0AF0040143
:101B10002C0E826FC5EC0AF01A0EE2EC08F0E8CF4A
:101B200000F11B0EE2EC08F0E8CF01F11C0EE2EC34
:101B300008F0E8CF02F11D0EE2EC08F0E8CF03F167
:101B400078EC13F004012C0E826FC5EC0AF092C100
:101B500000F193C101F194C102F195C103F178EC58
:101B600013F0CFEC0AF05DEF13F00401690E826F01
:101B7000C5EC0AF004012C0E826FC5EC0AF00101DD
:101B8000040E006F000E016F000E026F000E036F57
:101B900095EC19F02CC182F40401300E8227C5ECBB
:101BA0000AF02DC182F40401300E8227C5EC0AF040
:101BB0002EC182F40401300E8227C5EC0AF02FC139
:101BC00082F40401300E8227C5EC0AF030C182F4A1
:101BD0000401300E8227C5EC0AF031C182F4040101
:101BE000300E8227C5EC0AF032C182F40401300EB7
:101BF0008227C5EC0AF033C182F40401300E82273B
:101C0000C5EC0AF004012C0E826FC5EC0AF001014C
:101C1000030E006F000E016F000E026F000E036FC7
:101C200095EC19F02CC182F40401300E8227C5EC2A
:101C30000AF02DC182F40401300E8227C5EC0AF0AF
:101C40002EC182F40401300E8227C5EC0AF02FC1A8
:101C500082F40401300E8227C5EC0AF030C182F410
:101C60000401300E8227C5EC0AF031C182F4040170
:101C7000300E8227C5EC0AF032C182F40401300E26
:101C80008227C5EC0AF033C182F40401300E8227AA
:101C9000C5EC0AF004012C0E826FC5EC0AF00101BC
:101CA000280E006F000E016F000E026F000E036F12
:101CB00095EC19F02CC182F40401300E8227C5EC9A
:101CC0000AF02DC182F40401300E8227C5EC0AF01F
:101CD0002EC182F40401300E8227C5EC0AF02FC118
:101CE00082F40401300E8227C5EC0AF030C182F480
:101CF0000401300E8227C5EC0AF031C182F40401E0
:101D0000300E8227C5EC0AF032C182F40401300E95
:101D10008227C5EC0AF033C182F40401300E822719
:101D2000C5EC0AF004012C0E826FC5EC0AF0200EFF
:101D3000F86EF76AF66A04010900F5CF82F4C5EC83
:101D40000AF00900F5CF82F4C5EC0AF00900F5CFDE
:101D500082F4C5EC0AF00900F5CF82F4C5EC0AF074
:101D60000900F5CF82F4C5EC0AF00900F5CF82F442
:101D7000C5EC0AF00900F5CF82F4C5EC0AF00900C1
:101D8000F5CF82F4C5EC0AF0CFEC0AF05DEF13F06A
:101D90008351630AD8A45DEF13F08451610AD8A47B
:101DA0005DEF13F085516C0AD8A45DEF13F08651F6
:101DB000410A42E08651440A1BE08651420AD8B4E7
:101DC0002FEF0FF08651350AD8B4E7EF14F08651A3
:101DD000360AD8B43CEF15F08651370AD8B4A5EFCF
:101DE00015F08651380AD8B403EF16F05DEF13F002
:101DF0000798079A04017A0E826FC5EC0AF0040175
:101E0000780E826FC5EC0AF00401640E826FC5EC97
:101E10000AF081A813EF0FF00401550E826FC5EC94
:101E20000AF018EF0FF004014C0E826FC5EC0AF0B7
:101E3000CFEC0AF05DEF13F00788079A04017A0EE1
:101E4000826FC5EC0AF00401410E826FC5EC0AF006
:101E50000401610E826FC5EC0AF009EF0FF00798DC
:101E6000078A04017A0E826FC5EC0AF00401420E63
:101E7000826FC5EC0AF00401610E826FC5EC0AF0B6
:101E800009EF0FF0010166674DEF0FF067674DEF47
:101E90000FF068674DEF0FF0696765EF0FF04F6760
:101EA00059EF0FF0506759EF0FF0516759EF0FF0EE
:101EB000526765EF0FF00101000E006F000E016F19
:101EC000000E026F000E036F120011B873EF0FF0D7
:101ED0000101620E046F010E056F000E066F000E09
:101EE000076F7CEF0FF00101A70E046F020E056F64
:101EF000000E066F000E076F66C100F167C101F1A9
:101F000068C102F169C103F1F7EC18F003BFF7EF04
:101F10000FF00101000E046FA80E056F550E066F3D
:101F2000020E076F66C100F167C101F168C102F1DD
:101F300069C103F166C186F167C187F168C188F1A3
:101F400069C189F1F7EC18F003BFB0EF0FF00101A0
:101F5000000E866FA80E876F550E886F020E896F70
:101F60000E0EE2EC08F0E8CF18F10F0EE2EC08F0EC
:101F7000E8CF19F1100EE2EC08F0E8CF1AF1110EDB
:101F8000E2EC08F0E8CF1BF140EC18F086C104F158
:101F900087C105F188C106F189C107F1F7EC18F096
:101FA000078204EC18F040EC18F0079204EC18F0EB
:101FB00086C100F187C101F188C102F189C103F135
:101FC000079204EC18F0CC0E046FE00E056F870E3C
:101FD000066F050E076FF7EC18F000C118F101C18C
:101FE00019F102C11AF103C11BF12FEF10F0010129
:101FF000800E006F1A0E016F060E026F000E036F47
:102000004FC104F150C105F151C106F152C107F1B0
:10201000F7EC18F003AF10EF10F0F2EC19F012002B
:102020000E0EE2EC08F0E8CF18F10F0EE2EC08F02B
:10203000E8CF19F1100EE2EC08F0E8CF1AF1110E1A
:10204000E2EC08F0E8CF1BF14FC100F150C101F103
:1020500051C102F152C103F1078204EC18F018C11A
:1020600000F119C101F11AC102F11BC103F1120003
:102070000401730E826FC5EC0AF004012C0E826F0E
:10208000C5EC0AF0078462C166F163C167F164C1FF
:1020900068F165C169F14BC14FF14CC150F14DC1BF
:1020A00051F14EC152F157C159F158C15AF107943B
:1020B0005EEC10F0CFEC0AF05DEF13F066C100F1BA
:1020C00067C101F168C102F169C103F1010195EC39
:1020D00019F078EC17F00401630E826FC5EC0AF07A
:1020E00004012C0E826FC5EC0AF04FC100F150C103
:1020F00001F151C102F152C103F1010195EC19F056
:1021000078EC17F00401660E826FC5EC0AF004014A
:102110002C0E826FC5EC0AF0F2EC19F059C100F1F7
:102120005AC101F1010195EC19F078EC17F00401A6
:10213000740E826FC5EC0AF0120010820401530E77
:10214000826FC5EC0AF004012C0E826FC5EC0AF018
:1021500083C32AF184C32BF185C32CF186C32DF1EF
:1021600087C32EF188C32FF189C330F18AC331F1BF
:102170008BC332F18CC333F1010140EC1AF0B7ECA0
:1021800019F000C166F101C167F102C168F103C134
:1021900069F18EC32AF18FC32BF190C32CF191C347
:1021A0002DF192C32EF193C32FF194C330F195C357
:1021B00031F196C332F197C333F1010140EC1AF0CB
:1021C000B7EC19F000C14FF101C150F102C151F15A
:1021D00003C152F133EC1AF099C32FF19AC330F1D5
:1021E0009BC331F19CC332F19DC333F1010140EC3B
:1021F0001AF0B7EC19F000C159F101C15AF15EECC7
:1022000010F004012C0E826FC5EC0AF00FEF11F0F4
:102210008251520A03E10F820FEF11F00F928251A7
:10222000750A03E1108416EF11F0109411A01DEF50
:1022300011F011A41DEF11F010848251550A03E131
:10224000108624EF11F01096078410B281EF11F080
:1022500010A46DEF11F0B6C166F1B7C167F1B8C156
:1022600068F1B9C169F1BAC16AF1BBC16BF1BCC116
:102270006CF1BDC16DF1BEC16EF1BFC16FF1C0C1E6
:1022800070F1C1C171F1C2C172F1C3C173F1C4C1B6
:1022900074F1C5C175F1C6C176F1C7C177F1C8C186
:1022A00078F1C9C179F1CAC17AF1CBC17BF1CCC156
:1022B0007CF1CDC17DF1CEC17EF1CFC17FF1D0C126
:1022C00080F1D1C181F1D2C182F1D3C183F1D4C1F6
:1022D00084F1D5C185F175EF11F062C166F163C17A
:1022E00067F164C168F165C169F14BC14FF14CC13F
:1022F00050F14DC151F14EC152F157C159F158C180
:102300005AF107940FA0A3EF11F00101926790EF2B
:1023100011F0936790EF11F0946790EF11F09567CB
:1023200094EF11F0A3EF11F042EC0FF092C104F121
:1023300093C105F194C106F195C107F1F7EC18F0CE
:1023400003BF23EF13F042EC0FF00101000E046F06
:10235000000E056F010E066F000E076F28EC19F0D6
:1023600011A0E2EF11F011A2E2EF11F095EC19F0DB
:102370002967BDEF11F0C4EF11F004012D0E826F3B
:10238000C5EC0AF021EF13F030C182F40401300EE5
:102390008227C5EC0AF031C182F40401300E822795
:1023A000C5EC0AF032C182F40401300E8227C5EC7C
:1023B0000AF033C182F40401300E8227C5EC0AF022
:1023C00021EF13F010AEECEF11F095EC19F06EEC7C
:1023D0001AF0109E23EF13F010A4F6EF11F0040191
:1023E000750E826FC5EC0AF0FBEF11F00401720E5E
:1023F000826FC5EC0AF004012C0E826FC5EC0AF066
:1024000095EC19F029670AEF12F00401200E826F93
:102410000DEF12F004012D0E826FC5EC0AF030C1F1
:1024200082F40401300E8227C5EC0AF031C182F437
:102430000401300E8227C5EC0AF004012E0E826FD3
:10244000C5EC0AF032C182F40401300E8227C5ECDB
:102450000AF033C182F40401300E8227C5EC0AF081
:1024600004016D0E826FC5EC0AF004012C0E826F20
:10247000C5EC0AF04FC100F150C101F151C102F1A8
:1024800052C103F1010195EC19F078EC17F0040149
:10249000480E826FC5EC0AF004017A0E826FC5EC1B
:1024A0000AF004012C0E826FC5EC0AF066C100F13F
:1024B00067C101F168C102F169C103F1010195EC45
:1024C00019F078EC17F00401630E826FC5EC0AF086
:1024D00004012C0E826FC5EC0AF066C100F167C1E1
:1024E00001F168C102F169C103F101010A0E046F33
:1024F000000E056F000E066F000E076F08EC19F056
:10250000000E046F120E056F000E066F000E076FAF
:1025100028EC19F095EC19F02AC182F40401300E70
:102520008227C5EC0AF02BC182F40401300E822709
:10253000C5EC0AF02CC182F40401300E8227C5ECF0
:102540000AF02DC182F40401300E8227C5EC0AF096
:102550002EC182F40401300E8227C5EC0AF02FC18F
:1025600082F40401300E8227C5EC0AF030C182F4F7
:102570000401300E8227C5EC0AF004012E0E826F92
:10258000C5EC0AF031C182F40401300E8227C5EC9B
:102590000AF032C182F40401300E8227C5EC0AF041
:1025A00033C182F40401300E8227C5EC0AF0040125
:1025B000730E826FC5EC0AF004012C0E826FC5EC1D
:1025C0000AF0F2EC19F059C100F15AC101F187EC9F
:1025D00014F00FB2EFEF12F00FA021EF13F004018F
:1025E0002C0E826FC5EC0AF0200EF86EF76AF66AC0
:1025F00004010900F5CF82F4C5EC0AF00900F5CF1B
:1026000082F4C5EC0AF00900F5CF82F4C5EC0AF0BB
:102610000900F5CF82F4C5EC0AF00900F5CF82F489
:10262000C5EC0AF00900F5CF82F4C5EC0AF0090008
:10263000F5CF82F4C5EC0AF00900F5CF82F4C5ECC1
:102640000AF0CFEC0AF00F905DEF13F00401630E77
:10265000826FC5EC0AF004012C0E826FC5EC0AF003
:1026600063EC13F004012C0E826FC5EC0AF0D6EC7B
:1026700013F004012C0E826FC5EC0AF052EC14F03A
:1026800004012C0E826FC5EC0AF00101F80E006FF8
:10269000CD0E016F660E026F030E036F78EC13F020
:1026A00004012C0E826FC5EC0AF068EC14F0CFEC3C
:1026B0000AF05DEF13F0CFEC0AF00301C26B079054
:1026C00010926CEF16F0D8900E0EE2EC08F0E8CF06
:1026D00000F10F0EE2EC08F0E8CF01F1100EE2EC91
:1026E00008F0E8CF02F1110EE2EC08F0E8CF03F1B8
:1026F0000101000E046F000E056F010E066F000E43
:10270000076F28EC19F095EC19F02AC182F4040146
:10271000300E8227C5EC0AF02BC182F40401300E82
:102720008227C5EC0AF02CC182F40401300E822706
:10273000C5EC0AF02DC182F40401300E8227C5ECED
:102740000AF02EC182F40401300E8227C5EC0AF093
:102750002FC182F40401300E8227C5EC0AF030C18B
:1027600082F40401300E8227C5EC0AF031C182F4F4
:102770000401300E8227C5EC0AF004012E0E826F90
:10278000C5EC0AF032C182F40401300E8227C5EC98
:102790000AF033C182F40401300E8227C5EC0AF03E
:1027A00004016D0E826FC5EC0AF01200120EE2EC0D
:1027B00008F0E8CF00F1130EE2EC08F0E8CF01F1E9
:1027C000140EE2EC08F0E8CF02F1150EE2EC08F08E
:1027D000E8CF03F101010A0E046F000E056F000E31
:1027E000066F000E076F08EC19F0000E046F120E52
:1027F000056F000E066F000E076F28EC19F095ECC0
:1028000019F02AC182F40401300E8227C5EC0AF0C7
:102810002BC182F40401300E8227C5EC0AF02CC1D2
:1028200082F40401300E8227C5EC0AF02DC182F437
:102830000401300E8227C5EC0AF02EC182F4040197
:10284000300E8227C5EC0AF02FC182F40401300E4D
:102850008227C5EC0AF030C182F40401300E8227D1
:10286000C5EC0AF004012E0E826FC5EC0AF031C1EE
:1028700082F40401300E8227C5EC0AF032C182F4E2
:102880000401300E8227C5EC0AF033C182F4040142
:10289000300E8227C5EC0AF00401730E826FC5EC7E
:1028A0000AF012000A0EE2EC08F0E8CF00F10B0E7D
:1028B000E2EC08F0E8CF01F10C0EE2EC08F0E8CF12
:1028C00002F10D0EE2EC08F0E8CF03F187EF14F00F
:1028D000060EE2EC08F0E8CF00F1070EE2EC08F09B
:1028E000E8CF01F1080EE2EC08F0E8CF02F1090EA2
:1028F000E2EC08F0E8CF03F187EF14F00101F2EC0D
:1029000019F0078457C100F158C101F10794010182
:10291000E80E046F800E056F000E066F000E076F45
:1029200008EC19F0000E046F040E056F000E066F20
:10293000000E076F28EC19F0880E046F130E056F58
:10294000000E066F000E076FF7EC18F00A0E046F0A
:10295000000E056F000E066F000E076F28EC19F0D1
:1029600095EC19F001012967BBEF14F00401200E6A
:10297000826FBEEF14F004012D0E826FC5EC0AF0D9
:1029800030C182F40401300E8227C5EC0AF031C157
:1029900082F40401300E8227C5EC0AF032C182F4C1
:1029A0000401300E8227C5EC0AF004012E0E826F5E
:1029B000C5EC0AF033C182F40401300E8227C5EC65
:1029C0000AF00401430E826FC5EC0AF0120087C3BF
:1029D0002AF188C32BF189C32CF18AC32DF18BC353
:1029E0002EF18CC32FF18DC330F18EC331F190C322
:1029F00032F191C333F10101296B40EC1AF0B7ECCD
:102A000019F00101000E046F000E056F010E066F34
:102A1000000E076F08EC19F00E0E0C6E00C10BF0E3
:102A2000CBEC08F00F0E0C6E01C10BF0CBEC08F0F4
:102A3000100E0C6E02C10BF0CBEC08F0110E0C6EF8
:102A400003C10BF0CBEC08F004017A0E826FC5ECE9
:102A50000AF004012C0E826FC5EC0AF00401350E59
:102A6000826FC5EC0AF004012C0E826FC5EC0AF0EF
:102A700063EC13F018EF0FF087C32AF188C32BF132
:102A800089C32CF18AC32DF18BC32EF18CC32FF196
:102A90008DC330F18EC331F190C332F191C333F164
:102AA0000101296B40EC1AF0B7EC19F0880E046FA5
:102AB000130E056F000E066F000E076FFCEC18F08A
:102AC000000E046F040E056F000E066F000E076FF8
:102AD00008EC19F00101E80E046F800E056F000E7E
:102AE000066F000E076F28EC19F00A0E0C6E00C17D
:102AF0000BF0CBEC08F00B0E0C6E01C10BF0CBEC25
:102B000008F00C0E0C6E02C10BF0CBEC08F00D0EB1
:102B10000C6E03C10BF0CBEC08F004017A0E826F4F
:102B2000C5EC0AF004012C0E826FC5EC0AF004011A
:102B3000360E826FC5EC0AF004012C0E826FC5ECD4
:102B40000AF052EC14F018EF0FF087C32AF188C393
:102B50002BF189C32CF18AC32DF18BC32EF18CC3C9
:102B60002FF18DC330F18FC331F190C332F191C396
:102B700033F1010140EC1AF0B7EC19F0000E046FCC
:102B8000120E056F000E066F000E076F08EC19F0AD
:102B900001010A0E046F000E056F000E066F000E95
:102BA000076F28EC19F0120E0C6E00C10BF0CBEC85
:102BB00008F0130E0C6E01C10BF0CBEC08F0140EF4
:102BC0000C6E02C10BF0CBEC08F0150E0C6E03C1BD
:102BD0000BF0CBEC08F004017A0E826FC5EC0AF022
:102BE00004012C0E826FC5EC0AF00401370E826FCF
:102BF000C5EC0AF004012C0E826FC5EC0AF0D6EC8D
:102C000013F018EF0FF087C32AF188C32BF189C3A3
:102C10002CF18AC32DF18BC32EF18CC32FF18DC300
:102C200030F18EC331F190C332F191C333F1010120
:102C3000296B40EC1AF0B7EC19F0880E046F130EF4
:102C4000056F000E066F000E076FFCEC18F0000E0B
:102C5000046F040E056F000E066F000E076F08EC80
:102C600019F00101E80E046F800E056F000E066F6B
:102C7000000E076F28EC19F0060E0C6E00C10BF069
:102C8000CBEC08F0070E0C6E01C10BF0CBEC08F09A
:102C9000080E0C6E02C10BF0CBEC08F0090E0C6EA6
:102CA00003C10BF0CBEC08F004017A0E826FC5EC87
:102CB0000AF004012C0E826FC5EC0AF00401380EF4
:102CC000826FC5EC0AF004012C0E826FC5EC0AF08D
:102CD00068EC14F018EF0FF081A82AEF17F007A89E
:102CE000E3EF16F00101800E006F1A0E016F060E61
:102CF000026F000E036F4BC104F14CC105F14DC1D1
:102D000006F14EC107F1F7EC18F003BF2AEF17F0F8
:102D100072EC17F04BC100F14CC101F14DC102F151
:102D20004EC103F1078204EC18F018C104F119C177
:102D300005F11AC106F11BC107F1F80E006FCD0EA7
:102D4000016F660E026F030E036FF7EC18F00E0EA4
:102D50000C6E00C10BF0CBEC08F00F0E0C6E01C135
:102D60000BF0CBEC08F0100E0C6E02C10BF0CBECAC
:102D700008F0110E0C6E03C10BF0CBEC08F00784C9
:102D80000101F2EC19F057C100F158C101F10794AB
:102D90000A0E0C6E00C10BF0CBEC08F00B0E0C6EA3
:102DA00001C10BF0CBEC08F00C0E0C6E02C10BF065
:102DB000CBEC08F00D0E0C6E03C10BF0CBEC08F061
:102DC00007982AEF17F007AA2AEF17F007840101E6
:102DD000F2EC19F057C100F158C101F10794060E49
:102DE0000C6E00C10BF0CBEC08F0070E0C6E01C1AD
:102DF0000BF0CBEC08F0080E0C6E02C10BF0CBEC24
:102E000008F0090E0C6E03C10BF0CBEC08F0078440
:102E100062C100F163C101F164C102F165C103F156
:102E20000794120E0C6E00C10BF0CBEC08F0130EE1
:102E30000C6E01C10BF0CBEC08F0140E0C6E02C14D
:102E40000BF0CBEC08F0150E0C6E03C10BF0CBECC5
:102E500008F0079A0401805181197F0B0BE09EA8AE
:102E600009D014EE00F081517F0BE126E750812B51
:102E70000F01AD6E29EF0AF018C100F119C101F17F
:102E80001AC102F11BC103F1000E046F000E056FA1
:102E9000010E066F000E076F28EC19F029A167EFED
:102EA00017F02051D8B467EF17F018C100F119C11D
:102EB00001F11AC102F11BC103F1000E046F000EF3
:102EC000056F0A0E066F000E076F28EC19F012004E
:102ED000010104510013055101130651021307515A
:102EE000031312000101186B196B1A6B1B6B120094
:102EF0002AC182F40401300E8227C5EC0AF02BC1EE
:102F000082F40401300E8227C5EC0AF02CC182F451
:102F10000401300E8227C5EC0AF02DC182F40401B1
:102F2000300E8227C5EC0AF02EC182F40401300E67
:102F30008227C5EC0AF02FC182F40401300E8227EB
:102F4000C5EC0AF030C182F40401300E8227C5ECD2
:102F50000AF031C182F40401300E8227C5EC0AF078
:102F600032C182F40401300E8227C5EC0AF033C16D
:102F700082F40401300E8227C5EC0AF012002FC142
:102F800082F40401300E8227C5EC0AF030C182F4CD
:102F90000401300E8227C5EC0AF031C182F404012D
:102FA000300E8227C5EC0AF032C182F40401300EE3
:102FB0008227C5EC0AF033C182F40401300E822767
:102FC000C5EC0AF01200060E126E060E136E060E07
:102FD000146E122EE9EF17F0132EE9EF17F0142EEE
:102FE000E9EF17F08B84020E126E020E136E020EC2
:102FF000146E122EF9EF17F0132EF9EF17F0142EAE
:10300000F9EF17F08B9412000101005305E1015311
:1030100003E1025301E1002BC7EC18F0F2EC19F0C8
:103020003951006F3A51016F420E046F4B0E056F1C
:10303000000E066F000E076F08EC19F000C104F1D6
:1030400001C105F102C106F103C107F118C100F188
:1030500019C101F11AC102F11BC103F107B235EF29
:1030600018F0FCEC18F037EF18F0F7EC18F000C18E
:1030700018F101C119F102C11AF103C11BF11200CB
:10308000F2EC19F059C100F15AC101F1060EE2EC5F
:1030900008F0E8CF04F1070EE2EC08F0E8CF05F104
:1030A000080EE2EC08F0E8CF06F1090EE2EC08F0B9
:1030B000E8CF07F1F7EC18F000C124F101C125F1C8
:1030C00002C126F103C127F1290E046F000E056F1E
:1030D000000E066F000E076F08EC19F0EE0E046F7D
:1030E000430E056F000E066F000E076FFCEC18F024
:1030F00024C104F125C105F126C106F127C107F15C
:1031000008EC19F000C11CF101C11DF102C11EF152
:1031100003C11FF1120EE2EC08F0E8CF04F1130E28
:10312000E2EC08F0E8CF05F1140EE2EC08F0E8CF8D
:1031300006F1150EE2EC08F0E8CF07F10D0E006F76
:10314000000E016F000E026F000E036F08EC19F005
:10315000180E046F000E056F000E066F000E076F4D
:1031600028EC19F01CC104F11DC105F11EC106F1C6
:103170001FC107F1FCEC18F06A0E046F2A0E056FF0
:10318000000E066F000E076FF7EC18F01200BF0E6E
:10319000FA6E200E3A6F396BD8900037013702373C
:1031A0000337D8B0D8EF18F03A2FCDEF18F0390721
:1031B0003A070353D8B412000331070B80093F6F5D
:1031C00003390F0B010F396F80EC5FF0406F390549
:1031D00080EC5FF0405D405F396B3F33D8B03927FA
:1031E00039333FA9EDEF18F04051392712000101A2
:1031F00017EC1AF0D8B01200010103510719346F0F
:10320000DAEC19F0D8900751031934AF800F12008F
:103210000101346BFEEC19F0D8A014EC1AF0D8B010
:103220001200E9EC19F0F2EC19F01F0E366F2AECDF
:103230001AF00B35D8B0DAEC19F0D8A00335D8B0B5
:103240001200362F17EF19F034B101EC1AF012000A
:103250000101346B04510511061107110008D8A0B3
:10326000FEEC19F0D8A014EC1AF0D8B01200086BDC
:10327000096B0A6B0B6B2AEC1AF01F0E366F2AECE7
:103280001AF007510B5DD8A452EF19F006510A5DF0
:10329000D8A452EF19F00551095DD8A452EF19F0E6
:1032A0000451085DD8A065EF19F00451085F05517D
:1032B000D8A0053D095F0651D8A0063D0A5F075119
:1032C000D8A0073D0B5FD8900081362F3FEF19F053
:1032D00034B101EC1AF0346BFEEC19F0D8902EECFE
:1032E0001AF007510B5DD8A482EF19F006510A5D60
:1032F000D8A482EF19F00551095DD8A482EF19F026
:103300000451085DD8A091EF19F0003F91EF19F03A
:10331000013F91EF19F0023F91EF19F0032BD8B460
:10332000120034B101EC1AF012000101346BFEEC12
:1033300019F0D8B0120033EC1AF0200E366F0037B7
:1033400001370237033711EE33F00A0E376FE736D5
:103350000A0EE75CD8B0E76EE552372FA7EF19F0F9
:10336000362F9FEF19F034B12981D8901200010156
:103370000A0E346F200E366F11EE29F03451376F7C
:103380000A0ED890E652D8B0E726E732372FC2EFC0
:1033900019F00333023301330033362FBCEF19F039
:1033A000E750FF0FD8A00335D8B0120029B101ECC7
:1033B0001AF01200045100270551D8B0053D01272D
:1033C0000651D8B0063D02270751D8B0073D032764
:1033D00012000051086F0151096F02510A6F035129
:1033E0000B6F12000101006B016B026B036B12008B
:1033F0000101046B056B066B076B12000335D8A047
:1034000012000351800B001F011F021F031F003F0A
:1034100011EF1AF0013F11EF1AF0023F11EF1AF00D
:10342000032B342B032512000735D8A012000751B7
:10343000800B041F051F061F071F043F27EF1AF00C
:10344000053F27EF1AF0063F27EF1AF0072B342B22
:1034500007251200003701370237033708370937CD
:103460000A370B3712000101296B2A6B2B6B2C6B6F
:103470002D6B2E6B2F6B306B316B326B336B1200FD
:1034800001012A510F0B2A6F2B510F0B2B6F2C515F
:103490000F0B2C6F2D510F0B2D6F2E510F0B2E6F0D
:1034A0002F510F0B2F6F30510F0B306F31510F0B0E
:1034B000316F32510F0B326F33510F0B336F1200DC
:1034C0008194400EC76E220EC66E050EE82EFED702
:1034D00012008184050EE82EFED7120060EC1AF06F
:1034E0009E96C69E790EC96EFF0E9EB602D0E82E3D
:1034F000FCD79E96C69E000EC96EFF0E9EB602D0E9
:10350000E82EFCD70101306791EF1AF09E96C69E17
:10351000100EC96EFF0E9EB602D0E82EFCD79AEFB1
:103520001AF09E96C69E30C1C9FFFF0E9EB602D00D
:10353000E82EFCD79E96C69E31C1C9FFFF0E9EB6EF
:1035400002D0E82EFCD79E96C69E32C1C9FFFF0E60
:103550009EB602D0E82EFCD79E96C69E33C1C9FF08
:10356000FF0E9EB602D0E82EFCD769EC1AF01200CE
:1035700060EC1AF09E96C69E760EC96EFF0E9EB641
:1035800002D0E82EFCD769EC1AF060EC1AF09E9697
:10359000C69E770EC96EFF0E9EB602D0E82EFCD7EF
:1035A0009E96C69E020EC96EFF0E9EB602D0E82EF3
:1035B000FCD769EC1AF060EC1AF09E96C69E7A0E63
:1035C000C96EFF0E9EB602D0E82EFCD79E96C69E10
:1035D000550EC96EFF0E9EB602D0E82EFCD769ECE0
:0435E0001AF01200CB
:10BF0000E844F926000C160C2B0C3F0C520C640C68
:10BF1000760C860C960CA50CB30CC10CCF0CDC0C6B
:06BF2000E80CF40C000C1B
:00000001FF
